:0200000080245A
:1000230002017C1201069000511200991200B2D213
:01003300AF1D
:10003400D2AC75B0FF12016375995380FE3132332F
:0D0044003435363738393031323334353603
:100051004D6F64756C6F204141204C6973746F2141
:100061007F05000000000000DFF800227F0700008C
:100071000000000000000000DFF4000000227FE625
:10008100000000000000000000000000000000006F
:100091000000DFEC00000022C291D290781079FFBD
:1000A1000989E09385E080D291120061C291D8F074
:1000B10022C290C2917580C0D291120061C2912278
:1000C100C290C2918F80D287D291120061C29122D7
:1000D100C291D2907580FFD291120061C29122C269
:0100E100908E
:1000E200C291120061758080D291120061C2912288
:1000F200C291C290758001D29112007FC291D290BA
:1001020012007F22C290758038120061C291758000
:010112000FDD
:10011300D291120061C291758006D291120061C220
:01012300914A
:10012400758001D291120061C29112007F12007F8A
:1001340012007F12007FD29022EF75F00A844430BF
:1001440043F030C291D290F580D291120061C291F5
:10015400C291D29085F080D291120061C29122C2E4
:010164009901
:10016500C298D2AFD2ACC287758920758DFD758BCB
:01017500FD8C
:10017600D28E75985022209903209803C29932C2D4
:0101860098E0
:10018700E599F599C291D29085E080D291120061EC
:03019700C29132E0
:00000001FF
